:020000040000FA
:1000000083138316860185018509831207309F00BB
:1000100081218C217821A701A901A60AD1211720CD
:100020002E20AF204121BE20FF201C210D280F30A3
:10003000A00031308400000884038000840A840A10
:10004000A00B1B280F30A00041308400000884035F
:100050008000840A840AA00B262808003820A0000B
:100060000739A420BF00200E0739A420CF000800C4
:1000700026088207703400344034003400340034E1
:100080000034003445340034003400340034073484
:1000900000347034003400340034003455340034FB
:1000A00000340734503400340034703400340034E9
:1000B000003470347034703470340434403450344C
:1000C0000034003400340034403400340034003450
:1000D00000340734403407340034503400340034E2
:1000E00005340034003407340534003400347034EF
:1000F0000034003400347034703470340034003410
:1001000070347434753470347034703400340034A6
:10011000503407340034073450340034003445344C
:1001200054340734003400340034043400340034D0
:100130000034003400344534703470347534703415
:1001400074347034A6010800013E82070134013482
:100150000134013402340234043408340800051C2C
:10016000B820851CBB20A51C3016A5184016080019
:100170003016A51008004016A5140800A51CC320C1
:10018000A518CA200800B018D1283019D128B019F4
:10019000D1280800C018D1284019D128C019D12869
:1001A0000800D72125108030A300BF21D7212514B6
:1001B0004730A300BF21D7214130A300BF21D72161
:1001C0004D30A300BF21D7214530A300BF21D72147
:1001D0008830A300BF21D7214F30A300BF21D721F2
:1001E0005630A300BF21D7214530A300BF21D7211E
:1001F0005230A300BF212030A300BF21FE28A71B3F
:100200000B29051D04290800A7010F30A800A71716
:100210002713A5182717A70ADD2125102708A300F3
:10022000BF212514DD212D30A300BF21DD21A80B26
:100230000800A801A7010800A71F080027083F39E8
:10024000271F303E271B403E840080183B210019A9
:100250003B2180193B21840A80183B2100193B2156
:1002600080193B21840A840A80184021001940210A
:1002700080194021080080100011A713A90A080066
:10028000080025108030A300BF2125141030A000E5
:1002900030308400DD218830001888308018EF303D
:1002A0000019F2308019FF30001AF630A300BF2188
:1002B000840AA00B4A29DD212510C030A300BF21EC
:1002C00025141030A00040308400DD218830001853
:1002D00088308018EF300019F2308019FF30001A92
:1002E000F630A300BF21840AA00B6529DD21080098
:1002F000303084002030A0008001840AA00B7C29CB
:1003000008008316203098000730990083120730C8
:100310009F00903098000800D721D721D721D721FE
:1003200025103030A300B721D7213030A300B721EA
:10033000D7213030A300B721D7212030A300B72127
:10034000D7212830A300BF21D7210C30A300BF2123
:10035000D7210630A300BF21D7210130A300BF2140
:10036000D7210230A300BF21D7212514080023087C
:1003700086008611000006140000061008002308FD
:10038000F03986002518861506140610230EF0395C
:10039000A4002518A415240886000614061086114A
:1003A00008001430A000D721A00BD3290800643026
:1003B000A100DD21A10BD92908006430A200A20B05
:0403C000DF29080029
:02400E00023F6F
:00000001FF
